:100800008431512CFF3FFF3F7E14843120007F084C
:10081000FB000B1D1B2C85313825843120006D0B0E
:10082000122CED0102306D02031C182C0130ED0278
:10083000063095000B11911E2F2C0530FA00ED00AB
:1008400023001908FA007D08203E86000130870049
:100850007A0881000130FA00FD0720009112111E74
:10086000482C2100111E482C200065086602031840
:10087000462C6608203E86000130870001082300D0
:100880009A000130FA002000E607482C21001112DE
:100890002000111B1113911891107B08FF007E108E
:1008A00009008C31022C2000DF01210031083204C4
:1008B000031D5C2C01258431210034085402031DE2
:1008C000632C330853020318692C3408D40033080E
:1008D000D30000305402513003195302031C732C0F
:1008E0005030D300D4015408D6005308D50020005E
:1008F0005F080319842C5F08AE00AF012100D5000A
:1009000020002F082100D600210056085A02031D9E
:100910008B2C550859020318912C5A08D6005908F7
:10092000D500003056023330031955020318BB2C92
:1009300006302000A600A701210056082000A100D3
:10094000210055082000A0006430A200A3018B31D3
:100950000E23843120002108A9002008A800893135
:1009600099218431200027082100E4002000260876
:100970002100E300D02CD53086008701403F2000C5
:10098000AE00413FAF00AE35AF0DAE35AF0D2E0816
:10099000803E2100E300023020002F3D2100E400D2
:1009A000003056020530031955020318DE2C2500CD
:1009B00093012000EE156E088E000800F93020002B
:1009C0009B00210064082000AF0021006308200084
:1009D000AE002F0DAF0CAE0C2F0DAF0CAE0C2E08D1
:1009E0002500910003302100E3050030E4050430C8
:1009F000E335E40D890BF82C63080C3E25009300C9
:100A00000800E7302000670203181B2D21004D0865
:100A10002000A000DF00133067020318122D210010
:100A20005108182D8130670203181B2D21004F0833
:100A30002000A000DF00E730680203180800210052
:100A400049082000A000DF001330680203182E2D93
:100A5000210045082000A000DF0008008130680266
:100A600003180800210047082000A000DF0008004C
:100A7000F90120006C08790203186F2D7908F6003F
:100A80000130F635FF3E031D412D7635023E523EC4
:100A90008600013087000108F700F801F0007808AF
:100AA000F10021006608F3006508F2008025853119
:100AB00070087104031D6B2D7908F6000130F635BE
:100AC000FF3E031D5F2D7635033E523E860001300A
:100AD00087008101810A0130F600F907392D0130C4
:100AE0002100E5070030E63D27306602113003198A
:100AF0006502031C08000130E5000030E601080033
:100B0000700871040319A62DF501F50AF11B912D4A
:100B10000130F035F10D890B892D0130F400F50716
:100B2000862D71087302031D972D70087202031C35
:100B30009D2D7008F2027108F33B0130F136F00C84
:100B4000890B9E2D0130F502031D912D7308F100D4
:100B50007208F0000800220023082000B400B5014C
:100B6000220022082000B600B701B700B601340801
:100B70003604B90035083704BA00220025082000E1
:100B8000B400BB003A08A1003908A0003B08B4003B
:100B9000A20021002C088A002B080A0085312000C1
:100BA000B500BC003C08031DD82D02308B31DF2B73
:100BB0002000BD013B083D020318002E3D35083ED4
:100BC000203E8600013087000108B4003C08860002
:100BD0008701340881000130B400BC073D35073E71
:100BE000203E8600013087000108B4003C088600E2
:100BF0008701340881000130B400BC07BD07DA2D3D
:100C00000630A0018B312A23853108302000B40042
:100C1000E50055088A0054080A0086310800E030D3
:100C20002100AD000630AE00033020002102E83084
:100C300003192002031C362E22082007A3002108D6
:100C40000318210AA40003302402F0300319230200
:100C50000318362E2008183EA300A5000A302100F4
:100C6000DD00DE0120002535D33E080007302102DB
:100C7000D03003192002031C003422082007A300EF
:100C800021080318210AA40007302402E3300319C5
:100C900023020318003473302100AD000F30AE0082
:100CA00020002008303EA300A5002535AF3E0800F7
:100CB00021003D083E04031D9A2E2E3020006A02BA
:100CC0000318682E50302100D9000030DA010800E6
:100CD0004D3020006A020318732E3F302100D900E6
:100CE0000030DA010800803020006A0203187E2EEE
:100CF00020302100D9000030DA010800AE30200099
:100D00006A020318892E14302100D9000030DA015C
:100D10000800D13020006A020318942E0D30210003
:100D2000D9000030DA01080021003408DA00330865
:100D3000D90008003E08DA003D08D9000800230069
:100D40009D1CA92E1D122130890BA42E000023000A
:100D50001D16200065086602031C08006D08031DAF
:100D600008008A317822FD010800833408343234C7
:100D70000034B5340E34143400349F340634033454
:100D800000342000E601FD012100111623009E160B
:100D90000800FF34FF34FF34FF34FF3403340534DC
:100DA000FE0012001E00FE0BD12E003464008001F4
:100DB0000131890BD72E0034F4340134013400346E
:100DC0000800FF3FFF3FFF3FFF3FFF3FFF3FFF3F69
:10102000FF3FFF3FFF3FFF3FFF3FFF3FFF3F2200EC
:1010300023082000B400B501220022082000B600D9
:10104000B701B700B60134083604B90035083704D3
:10105000BA00220025082000B400BB00220025357C
:101060002000B4002200A20020003A08A1003908A4
:10107000A0003B08B400A20021002C088A002B0825
:101080000A0088312000B500BC003C08031D4A2836
:101090000230DF2B2000BD013B083D0203187228FF
:1010A0003C08860087010108B4003D35043E203E1F
:1010B000860001308700340881000130B400BC078D
:1010C0003C08860087010108B4003D35033E203E00
:1010D000860001308700340881000130B400BC076D
:1010E000BD074C28A00122002208033E2A2322002B
:1010F0002208053E2000B400E50055088A00540887
:101100000A0088310800063021002E06031D8A28B7
:10111000E0302D06031998288B132E088A002D081D
:101120000A0088318B17E0302100AD000630AE0098
:10113000ED218831CD2188312100A901AA0135088E
:101140003604031D1429FC302000A600A7016908FD
:10115000B000B101A0003108A1002100300820003A
:10116000A30021002F082000A2000E2388312000B8
:101170002108A9002008A80099218831200027080B
:10118000B5002608B40001303502003003193402DE
:10119000031CCD28FF30B400B5013408B0005A0854
:1011A000A03E860001308700300881000130B00089
:1011B000DA0714305A060319DA011430B201B30108
:1011C000B60136020318F6283608A03E8600013024
:1011D00087000108B000B101B2073108B33D01300A
:1011E000B000B60714303602031CE4281430A60001
:1011F000A7013308A9003208A800992188312000EE
:1012000027082100D400200026082100D30034083C
:101210005402031D0D2933085302031817293408FB
:10122000D4003308D30017298D31BF258831003011
:1012300021005402053003195302031822290330F8
:10124000A900AA0120006308031D2B2921005B18B7
:101250002B293A1F2F2903302100A900AA0186312A
:1012600058268831003021005A02053003195902EE
:10127000033003183D29A900AA0129062A04031DE9
:1012800059296D290130A9000030AA018B2188312C
:101290006D2902302100A9000030AA018B2188317C
:1012A0006D2902302100A9000030AA01F8238831FD
:1012B0006D2921005808003A03195F296D29570844
:1012C000013A03194229033A03194929013A03193A
:1012D0005129073A031951296D2921002A08E000F4
:1012E0002908DF005F03600403197B2903305F06D0
:1012F0006004031D8329250093012000EE156E086C
:101300008E008B218831023021005F066004031DAE
:1013100008008431532C2100611C0800FD3020009E
:10132000A000EE056E088E002100BA1A3A1761106F
:1013300008002000AB01AC01260827040319C829C6
:10134000AD01AD0AA71BAD290130A635A70D890B4C
:10135000A5290130AA00AD07A2290130AB35AC0D9B
:10136000890BAE2927082902031DB829260828025F
:10137000031CBF292608A8022708A93B2B1401300B
:10138000A736A60C890BC0290130AD02031DAD297B
:101390002C08A7002B08A6000800A03020006B0234
:1013A000031CDC2901302100D7000030D8012000C7
:1013B000E30121005B1008006F3020006B02031C6A
:1013C000E72902302100D7000030D801080003309F
:1013D0002100D7000030D80108002000FF30A20112
:1013E000A000A10021001D0883390C389D009D1428
:1013F0009D18F8291C082000A000E90021001D0804
:10140000833910389D009D149D18042A1C08200063
:10141000A000EA00210031083204031D242A1D081F
:10142000833904389D009D149D18142A1C0820003F
:10143000A000E800833021009D059D149D181E2A00
:101440001C082000A000E70020004130A501250273
:1014500003184A2A21001D08833908389D009D146D
:101460009D18302A1C082000A000A40022020318A6
:101470003C2A2408A000A200210824020318432AC1
:101480002408A000A1000130A000A50741302502DA
:10149000031C2A2A2208A0006408A03E86008701B7
:1014A000200881000130A000E4070530640603191C
:1014B000E4010530A301A50125020318742A2508BB
:1014C000A03E860087010108230203186D2A250823
:1014D000A03E86000108A000A3000130A000A507DF
:1014E00005302502031C5F2A2308A000EB0008003A
:1014F0002100310832040319080002307D02031C68
:101500000800103022002106031D932A2608093EF8
:101510002000BE00003003180130BF007D083E06E9
:101520003F04031D080008307D02031C0800210051
:1015300031082000BE00CC002200200820004C060C
:10154000031D08000330220021060319AD2A1030C4
:1015500021060319AD2A0130DF2B220025082000C7
:10156000BE00BF01220023082000C000C1012200EC
:1015700022082000C200C301A0004308A100FF30E0
:10158000A200A3010E238831200040082007C400D8
:101590004108213DC500220024082000C600C701E3
:1015A000A0004708A100FF30A200A3010E2388314C
:1015B000200020084407C8002108453DC9003E0816
:1015C0004807CA003F08493DCB001F304B0241305D
:1015D00003194A020318080022002408031D08000A
:1015E00015302502031808002000A001A00A7D087C
:1015F000FE3E2A238831003A03190C2B03302200C7
:101600002106031D052B17208831103022002106EA
:10161000031D08008531AB2D0830DF2B2000A4010D
:10162000A501201C172B2208A4072308A53D013083
:10163000A235A30D890B182B0130A136A00C890B04
:101640001D2B20082104031D112B2508A1002408AF
:10165000A00008002000AD00FF30B101B001AF00D4
:10166000AE00AB012D082B022E08A1002F08A2000E
:101670003008A3003108A4000318952B2B08203E46
:101680008600013087000108A500A601A701A80176
:10169000A1062608A2062708A3062808A4062408EF
:1016A000B1002308B0002208AF002108AE000830C6
:1016B000A100AC002C080319912B2E1C852B0130A6
:1016C000A100A030A200A301A4012E08A5002F08AC
:1016D000A6003008A7003108A8000130A836A70CE2
:1016E000A60CA50C890B6E2B2508A1062608A206C0
:1016F0002708A3062808A4062408B1002308B00080
:101700002208AF002108AE008C2B0130B136B00C9E
:10171000AF0CAE0C890B862B0130AC022C08031DDC
:101720005D2B0130A100AB07322B0830A436A30C8F
:10173000A20CA10C890B962B2108A5002508AA0054
:101740000830AE35AF0DB00DB10D890BA12B2E08B1
:10175000A1002F08A2003008A3003108A40008301F
:10176000A436A30CA20CA10C890BB02B2108A50058
:10177000A900200BCD2B2D08013E203E8600013014
:10178000870001082A06031D00342D08203E86002C
:10179000010829060319013400342908A1002D0885
:1017A000203E860001308700210881002A08A10020
:1017B0002D08013E203E86002108810001342000D2
:1017C000B3008030B2002200A10720003308B2002D
:1017D0002200A20020000330A0012A2305302000AF
:1017E000B200E50055088A0054080A008B31080051
:1017F00021006118FF2B2000EE146E088E002100DE
:1018000061140800C9308400863085006730860086
:101810000030870007308631D0268C31DC308400E0
:1018200086308500E3308600003087000430863142
:10183000D0268C31B5308400863085005230860049
:10184000013087000C308631D0268C31FC01FD013F
:10185000503084000030850017308631D6268C3118
:10186000A03084000030850043308631D6268C318C
:10187000203084000130850032308631D6268C310C
:10188000A03084000130850014308631D6268C319A
:101890007E1020004B2C6A3021009900FF308C0014
:1018A000E1308E0008302000CF00EE008E00603066
:1018B00021009E001D141D08833908389D00250055
:1018C000161522001E1101302100950024000C1471
:1018D0008C140C118C110C168C120E101A258C31D4
:1018E00021001708C13916389700171439278C3191
:1018F00020000030D001D1015102053003195002FF
:101900000318942CFF30CF005008A03E86008701BA
:101910004F0881000130D0070030D13D5102053021
:1019200003195002031C822C210031083204031DCC
:10193000E52C20000930D001D1015102C430031937
:1019400050020318DD2C21001D0883390C389D003E
:101950009D149D18A92C1C082000CF00E9003230EE
:10196000690256080318BF2C031DBE2C0130CF009E
:10197000D70740278C312000D601D60A5608031914
:10198000CC2C65306902031CCC2C0130CF00D7076A
:1019900039278C312000D6016400BE300032890B1B
:1019A000CE2C01302000D0070030D13D093051024B
:1019B000C43003195002031CA32C0A305702031C25
:1019C000E52C01302100B100B20140278C31C1303B
:1019D0002000D4000630D5000F302100AB000630C7
:1019E000AC00E030AD000630AE003108320403191F
:1019F000FB2C76258C318B170B17210091148B163D
:101A0000053020009C0021003008D4002F08D300AE
:101A1000FD30D701D80161102000CF00EE056E081F
:101A20008E0001302100DF000030E000BA13852570
:101A30008C31172DAF302000AB00AD002530AE014A
:101A40002E020318362D2E0867258C312000AB009E
:101A50002E082D07AC00860087012B08810001307D
:101A6000AB00AE0725302E02031C232D2100430FAF
:101A70000800440F08002030AF000530B001B1016C
:101A8000B201B3000130B401B500B601B701B8012D
:101A9000B9000630BA01BB01BC01BD01BE01C300E3
:101AA0000A30C401C5001030C601C7001930C80192
:101AB000C9002030CA01CB003030CC01CD003F300E
:101AC000CE01CF005030D001D100D201732F2000C1
:101AD000A200A000A1012300910020002108230002
:101AE00092009513151315141308080022009D1772
:101AF0001D1523001E159C0119309B001E129D17F9
:101B00001D168C102100911608002000CE016C08D3
:101B10004E02031808004E08CD000130CD35FF3EBF
:101B2000031D8E2D4D35033E523E86000130870049
:101B300001080319BB2D4E08CD000130CD35FF3E05
:101B4000031D9E2D4D35523E860001308700413FDA
:101B50008A00403F0A008D3120004E08CD00013040
:101B6000CD35FF3E031DB02D4D35033E523E860060
:101B70000130870081010130CD00CE07872D323042
:101B80002000690200300318792E53020B3003192C
:101B90005202031CD72D2100B91CD72D0330570644
:101BA0005804031DD72D2000E301E30A080021009B
:101BB000391C08000030200053021F300319520264
:101BC000031C732E1F3052065304031D0C2E1430B9
:101BD000D801D901DE015E0203180C2E39278C31A1
:101BE0000D302000A600FB30890BF42DA60BF42D40
:101BF000003240278C310D302000A600FB30890BCD
:101C0000FF2DA60BFF2D003201302000A600DE07BD
:101C100014305E02031CEE2D0630A000A101530813
:101C2000A3005208A20047278C3104302000200670
:101C30002104031D632E21003508360403192B2EC1
:101C4000003036020B300319350203182B2E3508ED
:101C50002000A600D8070B30210035063604031DEE
:101C60003D2E09302000590203183D2E5935C33E40
:101C7000860087010108A600D80020005808A600A9
:101C8000A7012100340820002702031D4B2E21004C
:101C90003308200026020318532E21003408D400F4
:101CA0003308D3005D2E20005808A600A7012100AC
:101CB000D300200027082100D40001302000A60016
:101CC000D90739278C3106302000A000A101530824
:101CD000A3005208A20047278C31200020082104CD
:101CE000031D732E402701302000D2070030D33D62
:101CF000080053021F3003195202031CB22E143085
:101D0000DE015E020318A22E39278C310D3020002F
:101D1000A600FB30890B8A2EA60B8A2E00324027A4
:101D20008C310D302000A600FB30890B952EA60BC0
:101D3000952E003201302000A600DE0714305E022E
:101D4000031C842E2100370838040319AF2E5408D1
:101D5000B0005308AF007330AD000F30AE0020006C
:101D6000D201D301D201D301080020006208031977
:101D7000640021003A1BCF2EEF2E39278C31E42E40
:101D800040278C31E42E39278C31E42E40278C31CA
:101D9000E42E39278C31E42E40278C31E42E2000AC
:101DA0005B08013A0319BD2E053A0319C02E033A08
:101DB0000319C32E0D3A0319C62E073A0319C92E6B
:101DC0001D3A0319CC2EE42E333020005B02031C95
:101DD000EB2EDB0108000130A100DB07080020002A
:101DE00052085304031D0800210057035804031D23
:101DF000032F7C08031DFF2E39278C31032F7C0B0A
:101E0000032F40278C310230210057065804031D50
:101E10001F2F7C08031D0F2F39278C311F2F7C0BA0
:101E2000122F1D2F05307C06031D192F39278C31E9
:101E30001F2F06307C06031D1F2F40278C310330D7
:101E4000210057065804031D302F7C08031D2B2F3B
:101E500039278C31302F0A307C06031D302F402764
:101E600001302000A100FC0715307C020318FC01A2
:101E7000080014302000A000EE046E088E00080058
:101E8000EB302000A000EE056E088E000800200058
:101E90002008210403196E2FA501A50AA11B592FA3
:101EA0000130A035A10D890B512F0130A400A507E9
:101EB0004E2F21082302031D5F2F20082202031C3E
:101EC000652F2008A2022108A33B0130A136A00CF7
:101ED000890B662F0130A502031D592F2308A1008D
:101EE0002208A0000800AF302000A500A90024307F
:101EF000A500A800003021003002513003192F0244
:101F0000031C852F5030AF00B001003034020E307A
:101F100003193302031C8F2F0530B300B4013408BA
:101F20003002031D952F33082F0203189B2F34080E
:101F3000B0003308AF00003036020C300319350210
:101F4000031CA52F0130B500B6012000AA01280806
:101F50002A020318C92F2A0867258C312000A50002
:101F6000A7002A082907A50086008701010827067F
:101F70000319C42F2A082907A50086000108A60016
:101F8000A0002A08D0278C3101302000A500AA0724
:101F9000A72F2100BA1F08002000E201E20A080072
:101FA0002000A300A100A20123009100200022082C
:101FB000230092002000200823009300951315139E
:101FC00015150B082000A100A4008B01553023003B
:101FD0009600AA3096009514200024088B00033048
:101FE000890BF02F00002000121AFB2F0330890B01
:101FF000F72F0000F32F2300151120001212080004
:020000040001F9
:04000E00BCF9FFDE5C
:00000001FF
